 buspcie950

 Timestamp is 494a89f5 (Thu Dec 18 17:35:49 2008)

 Preferred load address is 10000000

 Start         Length     Name                   Class
 0001:00000000 00000a36H .rdata                  CODE
 0001:00000a38 0000005dH .rdata$debug            CODE
 0001:00000a98 000025f0H .text                   CODE
 0001:00003088 00000028H .idata$2                CODE
 0001:000030b0 00000014H .idata$3                CODE
 0001:000030c4 000000a8H .idata$4                CODE
 0001:0000316c 00000016H .idata$6                CODE
 0001:00003190 00000057H .edata                  CODE
 0002:00000000 000000a8H .idata$5                DATA
 0002:000000a8 00000444H .data                   DATA
 0002:00000500 00000120H .bss                    DATA
 0003:00000000 00000070H .pdata                  DATA

  Address         Publics by Value              Rva+Base     Lib:Object

 0000:00000000       ___safe_se_handler_table   00000000     <absolute>
 0000:00000000       ___safe_se_handler_count   00000000     <absolute>
 0001:0000001c       ??_C@_19OBNDINH@?$AAP?$AAo?$AAr?$AAt?$AA?$AA@ 1000101c     buspcie950.obj
 0001:00000028       ??_C@_1BI@IGMEDLLH@?$AA?$CF?$AAs?$AA?2?$AAU?$AAn?$AAi?$AAm?$AAo?$AAd?$AAe?$AAm?$AA?$AA@ 10001028     buspcie950.obj
 0001:00000040       ??_C@_1BK@BFIEKNFP@?$AAF?$AAr?$AAi?$AAe?$AAn?$AAd?$AAl?$AAy?$AAN?$AAa?$AAm?$AAe?$AA?$AA@ 10001040     buspcie950.obj
 0001:0000005c       ??_C@_1BG@KCOOGCNN@?$AAD?$AAe?$AAv?$AAi?$AAc?$AAe?$AAT?$AAy?$AAp?$AAe?$AA?$AA@ 1000105c     buspcie950.obj
 0001:00000074       ??_C@_1BK@HFHDBJKI@?$AAU?$AAn?$AAi?$AAm?$AAo?$AAd?$AAe?$AAm?$AA?4?$AAd?$AAl?$AAl?$AA?$AA@ 10001074     buspcie950.obj
 0001:00000090       ??_C@_19LJDFFCJJ@?$AA?$CF?$AAs?$AA?$CF?$AAs?$AA?$AA@ 10001090     buspcie950.obj
 0001:0000009c       ??_C@_1BO@DLFIJDKP@?$AA?$CF?$AAs?$AA?2?$AAS?$AAe?$AAr?$AAi?$AAa?$AAl?$AAC?$AAa?$AAb?$AAl?$AAe?$AA?$AA@ 1000109c     buspcie950.obj
 0001:000000bc       ??_C@_1O@OFBIJOJC@?$AA?$CF?$AAs?$AA?$CF?$AA0?$AA2?$AAd?$AA?$AA@ 100010bc     buspcie950.obj
 0001:000000cc       ??_C@_1CA@INOAHGHF@?$AAB?$AAu?$AAs?$AAA?$AAc?$AAc?$AAe?$AAs?$AAs?$AAH?$AAa?$AAn?$AAd?$AAl?$AAe?$AA?$AA@ 100010cc     buspcie950.obj
 0001:000000ec       ??_C@_1O@GBAEOCCH@?$AAP?$AAr?$AAe?$AAf?$AAi?$AAx?$AA?$AA@ 100010ec     buspcie950.obj
 0001:000000fc       ??_C@_1BE@GPBAGNPC@?$AAI?$AAs?$AAr?$AAH?$AAa?$AAn?$AAd?$AAl?$AAe?$AA?$AA@ 100010fc     buspcie950.obj
 0001:00000110       ??_C@_1BC@MCDIKBIL@?$AAI?$AAs?$AAt?$AAE?$AAv?$AAe?$AAn?$AAt?$AA?$AA@ 10001110     buspcie950.obj
 0001:00000124       ??_C@_1BG@LJAMCNJN@?$AAP?$AAo?$AAr?$AAt?$AAN?$AAu?$AAm?$AAb?$AAe?$AAr?$AA?$AA@ 10001124     buspcie950.obj
 0001:0000013c       ??_C@_1CC@KMPFMANC@?$AAD?$AAe?$AAv?$AAi?$AAc?$AAe?$AAA?$AAr?$AAr?$AAa?$AAy?$AAI?$AAn?$AAd?$AAe?$AAx?$AA?$AA@ 1000113c     buspcie950.obj
 0001:00000160       ??_C@_17DJMMGLBL@?$AAD?$AAl?$AAl?$AA?$AA@ 10001160     buspcie950.obj
 0001:00000168       ??_C@_19DIEFAIMH@?$AAC?$AAM?$AA?$CF?$AAd?$AA?$AA@ 10001168     buspcie950.obj
 0001:00000174       ??_C@_1M@OAJFFPML@?$AAF?$AAl?$AAa?$AAg?$AAs?$AA?$AA@ 10001174     buspcie950.obj
 0001:00000180       ??_C@_1BE@EODMIMC@?$AA?$CF?$AAs?$AA?2?$AAp?$AAo?$AAr?$AAt?$AA?$CF?$AAd?$AA?$AA@ 10001180     buspcie950.obj
 0001:00000194       ??_C@_15KOIPKGHO@?$AAC?$AAM?$AA?$AA@ 10001194     buspcie950.obj
 0001:0000019c       ??_C@_17KKLPNNMB@?$AAC?$AAO?$AAM?$AA?$AA@ 1000119c     buspcie950.obj
 0001:000001a4       ??_C@_1CE@HBCGCCG@?$AAD?$AAr?$AAi?$AAv?$AAe?$AAr?$AAs?$AA?2?$AAA?$AAc?$AAt?$AAi?$AAv?$AAe?$AA?2?$AA?$CF?$AAs?$AA?$AA@ 100011a4     buspcie950.obj
 0001:000001c8       ??_C@_19DINFBLAK@?$AAN?$AAa?$AAm?$AAe?$AA?$AA@ 100011c8     buspcie950.obj
 0001:000001d4       ??_C@_1BO@JJBEOHCE@?$AAD?$AAr?$AAi?$AAv?$AAe?$AAr?$AAs?$AA?2?$AAA?$AAc?$AAt?$AAi?$AAv?$AAe?$AA?$AA@ 100011d4     buspcie950.obj
 0001:000001f4       ??_C@_1CM@HIMBKDJM@?$AAL?$AAi?$AAn?$AAe?$AAD?$AAr?$AAi?$AAv?$AAe?$AAr?$AAD?$AAe?$AAl?$AAa?$AAy?$AAP?$AAh?$AAa?$AAs?$AAe@ 100011f4     buspcie950.obj
 0001:00000220       ??_C@_1CI@GLAIJPLJ@?$AAL?$AAi?$AAn?$AAe?$AAD?$AAr?$AAi?$AAv?$AAe?$AAr?$AAD?$AAe?$AAl?$AAa?$AAy?$AAB?$AAi?$AAt?$AAs?$AA?$AA@ 10001220     buspcie950.obj
 0001:00000248       ??_C@_1CI@OJPKJBA@?$AAB?$AAa?$AAu?$AAd?$AAr?$AAa?$AAt?$AAe?$AAM?$AAa?$AAp?$AAL?$AAi?$AAs?$AAt?$AAF?$AAr?$AAo?$AAm?$AA?$AA@ 10001248     buspcie950.obj
 0001:00000270       ??_C@_1CE@BHEKDMEI@?$AAB?$AAa?$AAu?$AAd?$AAr?$AAa?$AAt?$AAe?$AAM?$AAa?$AAp?$AAL?$AAi?$AAs?$AAt?$AAT?$AAo?$AA?$AA@ 10001270     buspcie950.obj
 0001:00000294       ??_C@_1BE@DDEHHBPD@?$AAD?$AAe?$AAv?$AAC?$AAo?$AAn?$AAf?$AAi?$AAg?$AA?$AA@ 10001294     buspcie950.obj
 0001:000002a8       ??_C@_17KNDIACFJ@?$AAT?$AAs?$AAp?$AA?$AA@ 100012a8     buspcie950.obj
 0001:000002b0       ??_C@_1BG@JDAFHBOG@?$AAI?$AAS?$AAR?$AAH?$AAa?$AAn?$AAd?$AAl?$AAe?$AAr?$AA?$AA@ 100012b0     buspcie950.obj
 0001:000002c8       ??_C@_1BG@NELPJJNN@?$AAI?$AAs?$AAr?$AAH?$AAa?$AAn?$AAd?$AAl?$AAe?$AAr?$AA?$AA@ 100012c8     buspcie950.obj
 0001:000002e0       ??_C@_1BO@KACPNJCM@?$AAi?$AAs?$AAr?$AAp?$AAc?$AAi?$AAe?$AA9?$AA5?$AA0?$AA?4?$AAd?$AAl?$AAl?$AA?$AA@ 100012e0     buspcie950.obj
 0001:00000300       ??_C@_1O@MDNCMDKF@?$AAI?$AAs?$AAr?$AAD?$AAl?$AAl?$AA?$AA@ 10001300     buspcie950.obj
 0001:00000310       ??_C@_1BO@NHAHMBJD@?$AAc?$AAo?$AAm?$AAp?$AAc?$AAi?$AAe?$AA9?$AA5?$AA0?$AA?4?$AAd?$AAl?$AAl?$AA?$AA@ 10001310     buspcie950.obj
 0001:00000330       ??_C@_1BA@CEFELOID@?$AAU?$AAa?$AAr?$AAt?$AAD?$AAl?$AAl?$AA?$AA@ 10001330     buspcie950.obj
 0001:00000340       ??_C@_1BA@BDHDGOBO@?$AAS?$AAy?$AAs?$AAI?$AAn?$AAt?$AAr?$AA?$AA@ 10001340     buspcie950.obj
 0001:00000350       ??_C@_17DJGGJCGD@?$AAI?$AAr?$AAq?$AA?$AA@ 10001350     buspcie950.obj
 0001:00000358       ??_C@_1BM@MHMIAMLB@?$AAI?$AAn?$AAt?$AAe?$AAr?$AAf?$AAa?$AAc?$AAe?$AAT?$AAy?$AAp?$AAe?$AA?$AA@ 10001358     buspcie950.obj
 0001:00000374       ??_C@_1BE@MNDDMKMB@?$AAB?$AAu?$AAs?$AAN?$AAu?$AAm?$AAb?$AAe?$AAr?$AA?$AA@ 10001374     buspcie950.obj
 0001:00000388       ??_C@_1O@LBBNFMDB@?$AAM?$AAe?$AAm?$AAL?$AAe?$AAn?$AA?$AA@ 10001388     buspcie950.obj
 0001:00000398       ??_C@_1BA@INLDIDEN@?$AAM?$AAe?$AAm?$AAB?$AAa?$AAs?$AAe?$AA?$AA@ 10001398     buspcie950.obj
 0001:000003a8       ??_C@_1M@PEPOCCHH@?$AAI?$AAo?$AAL?$AAe?$AAn?$AA?$AA@ 100013a8     buspcie950.obj
 0001:000003b4       ??_C@_1O@JMCNHCBG@?$AAI?$AAo?$AAB?$AAa?$AAs?$AAe?$AA?$AA@ 100013b4     buspcie950.obj
 0001:000003c4       ??_C@_1CE@PJBMNJAF@?$AAL?$AAi?$AAn?$AAe?$AAD?$AAr?$AAi?$AAv?$AAe?$AAr?$AAC?$AAo?$AAn?$AAt?$AAr?$AAo?$AAl?$AA?$AA@ 100013c4     buspcie950.obj
 0001:000003e8       ??_C@_1CE@HLGCKFJ@?$AAF?$AAl?$AAo?$AAw?$AAC?$AAt?$AAr?$AAl?$AAH?$AAi?$AAg?$AAh?$AAL?$AAe?$AAv?$AAe?$AAl?$AA?$AA@ 100013e8     buspcie950.obj
 0001:0000040c       ??_C@_1CC@ELLFOF@?$AAF?$AAl?$AAo?$AAw?$AAC?$AAt?$AAr?$AAl?$AAL?$AAo?$AAw?$AAL?$AAe?$AAv?$AAe?$AAl?$AA?$AA@ 1000140c     buspcie950.obj
 0001:00000430       ??_C@_1BO@MCGADMLE@?$AAR?$AAx?$AAI?$AAn?$AAt?$AAT?$AAr?$AAi?$AAg?$AAL?$AAe?$AAv?$AAe?$AAl?$AA?$AA@ 10001430     buspcie950.obj
 0001:00000450       ??_C@_1BO@ELCCHGIE@?$AAT?$AAx?$AAI?$AAn?$AAt?$AAT?$AAr?$AAi?$AAg?$AAL?$AAe?$AAv?$AAe?$AAl?$AA?$AA@ 10001450     buspcie950.obj
 0001:00000470       ??_C@_1CC@EKOCNIBB@?$AAC?$AAr?$AAy?$AAs?$AAt?$AAa?$AAl?$AAF?$AAr?$AAe?$AAq?$AAu?$AAe?$AAn?$AAc?$AAy?$AA?$AA@ 10001470     buspcie950.obj
 0001:00000494       ??_C@_1BK@KAMHHDIE@?$AAB?$AAr?$AAa?$AAn?$AAd?$AAi?$AAn?$AAg?$AAF?$AAi?$AAl?$AAe?$AA?$AA@ 10001494     buspcie950.obj
 0001:000004b0       ??_C@_1BM@CMGCPMHF@?$AAR?$AAe?$AAa?$AAd?$AAB?$AAr?$AAa?$AAn?$AAd?$AAF?$AAi?$AAl?$AAe?$AA?$AA@ 100014b0     buspcie950.obj
 0001:000004cc       ??_C@_17KACEIPNC@?$AAK?$AAe?$AAy?$AA?$AA@ 100014cc     buspcie950.obj
 0001:000004d4       ??_C@_1CC@KACJOILC@?$AAS?$AAe?$AAr?$AAi?$AAa?$AAl?$AA?5?$AAC?$AAa?$AAb?$AAl?$AAe?$AA?5?$AAo?$AAn?$AA?5?$AA?$AA@ 100014d4     buspcie950.obj
 0001:000004f8       ??_C@_1CK@MHPGFJDK@?$AAH?$AAa?$AAy?$AAe?$AAs?$AA?5?$AAC?$AAo?$AAm?$AAp?$AAa?$AAt?$AAi?$AAb?$AAl?$AAe?$AA?5?$AAo?$AAn?$AA?5@ 100014f8     buspcie950.obj
 0001:00000524       ??_C@_1M@FFLAJJMG@?$AA?$DM?$AAE?$AAN?$AAD?$AA?$DO?$AA?$AA@ 10001524     ConfigParser.obj
 0001:00000530       ??_C@_1CG@LGKPGFHM@?$AAN?$AAo?$AA?5?$AAC?$AAo?$AAn?$AAt?$AAr?$AAo?$AAl?$AA?5?$AA?$CI?$AAR?$AAS?$AA2?$AA3?$AA2?$AA?$CJ?$AA?$AA@ 10001530     ConfigParser.obj
 0001:00000558       ??_C@_1CO@KJKNEDLA@?$AAL?$AAo?$AAw?$AA?5?$AAE?$AAn?$AAa?$AAb?$AAl?$AAe?$AA?5?$AA?$CI?$AAR?$AAS?$AA4?$AA2?$AA2?$AA?1?$AA4?$AA8@ 10001558     ConfigParser.obj
 0001:00000588       ??_C@_1BI@LGOMGNKN@?$AAH?$AAi?$AAg?$AAh?$AA?5?$AAE?$AAn?$AAa?$AAb?$AAl?$AAe?$AA?$AA@ 10001588     ConfigParser.obj
 0001:000005a0       ??_C@_19BIEPDBPA@?$AAT?$AAy?$AAp?$AAe?$AA?$AA@ 100015a0     ConfigParser.obj
 0001:000005ac       ??_C@_1CI@IMABDCBP@?$AAL?$AAi?$AAn?$AAe?$AA_?$AAD?$AAr?$AAi?$AAv?$AAe?$AAr?$AA_?$AAC?$AAo?$AAn?$AAt?$AAr?$AAo?$AAl?$AA?$AA@ 100015ac     ConfigParser.obj
 0001:000005d4       ??_C@_1BK@CENGCIFF@?$AAT?$AAo?$AA_?$AAB?$AAa?$AAu?$AAd?$AA_?$AAR?$AAa?$AAt?$AAe?$AA?$AA@ 100015d4     ConfigParser.obj
 0001:000005f0       ??_C@_1BO@CILDMCD@?$AAF?$AAr?$AAo?$AAm?$AA_?$AAB?$AAa?$AAu?$AAd?$AA_?$AAR?$AAa?$AAt?$AAe?$AA?$AA@ 100015f0     ConfigParser.obj
 0001:00000610       ??_C@_1CC@FHAFLLA@?$AAB?$AAa?$AAu?$AAd?$AAr?$AAa?$AAt?$AAe?$AA_?$AAM?$AAa?$AAp?$AAp?$AAi?$AAn?$AAg?$AA?$AA@ 10001610     ConfigParser.obj
 0001:00000634       ??_C@_1BE@GELDBLFK@?$AAT?$AAa?$AAb?$AA_?$AAA?$AAb?$AAo?$AAu?$AAt?$AA?$AA@ 10001634     ConfigParser.obj
 0001:00000648       ??_C@_1DA@NCKAKAMN@?$AAT?$AAa?$AAb?$AA_?$AAL?$AAi?$AAn?$AAe?$AA_?$AAD?$AAr?$AAi?$AAv?$AAe?$AAr?$AA_?$AAC?$AAo?$AAn?$AAt@ 10001648     ConfigParser.obj
 0001:00000678       ??_C@_1CA@LJNFGPHD@?$AAT?$AAa?$AAb?$AA_?$AAF?$AAi?$AAf?$AAo?$AA_?$AAL?$AAe?$AAv?$AAe?$AAl?$AAs?$AA?$AA@ 10001678     ConfigParser.obj
 0001:00000698       ??_C@_1CK@NLOLPFMM@?$AAT?$AAa?$AAb?$AA_?$AAB?$AAa?$AAu?$AAd?$AAr?$AAa?$AAt?$AAe?$AA_?$AAM?$AAa?$AAp?$AAp?$AAi?$AAn?$AAg@ 10001698     ConfigParser.obj
 0001:000006c4       ??_C@_1CM@OFMOCLCD@?$AAT?$AAa?$AAb?$AA_?$AAC?$AAr?$AAy?$AAs?$AAt?$AAa?$AAl?$AA_?$AAF?$AAr?$AAe?$AAq?$AAu?$AAe?$AAn?$AAc@ 100016c4     ConfigParser.obj
 0001:000006f0       ??_C@_1BI@LMBHJBLG@?$AAT?$AAa?$AAb?$AA_?$AAO?$AAp?$AAt?$AAi?$AAo?$AAn?$AAs?$AA?$AA@ 100016f0     ConfigParser.obj
 0001:00000708       ??_C@_1DG@MMINKBLM@?$AAF?$AAl?$AAo?$AAw?$AA_?$AAC?$AAo?$AAn?$AAt?$AAr?$AAo?$AAl?$AA_?$AAO?$AAf?$AAf?$AA_?$AAL?$AAe?$AAv@ 10001708     ConfigParser.obj
 0001:00000740       ??_C@_1DG@FFKMCLJC@?$AAF?$AAl?$AAo?$AAw?$AA_?$AAC?$AAo?$AAn?$AAt?$AAr?$AAo?$AAl?$AA_?$AAO?$AAf?$AAf?$AA_?$AAL?$AAe?$AAv@ 10001740     ConfigParser.obj
 0001:00000778       ??_C@_1DE@JAENBBJL@?$AAF?$AAl?$AAo?$AAw?$AA_?$AAC?$AAo?$AAn?$AAt?$AAr?$AAo?$AAl?$AA_?$AAO?$AAn?$AA_?$AAL?$AAe?$AAv?$AAe@ 10001778     ConfigParser.obj
 0001:000007ac       ??_C@_1DE@JGMJLLF@?$AAF?$AAl?$AAo?$AAw?$AA_?$AAC?$AAo?$AAn?$AAt?$AAr?$AAo?$AAl?$AA_?$AAO?$AAn?$AA_?$AAL?$AAe?$AAv?$AAe@ 100017ac     ConfigParser.obj
 0001:000007e0       ??_C@_1DO@FFHHIFI@?$AAR?$AAx?$AA_?$AAI?$AAn?$AAt?$AAe?$AAr?$AAr?$AAu?$AAp?$AAt?$AA_?$AAT?$AAr?$AAi?$AAg?$AAg?$AAe?$AAr@ 100017e0     ConfigParser.obj
 0001:00000820       ??_C@_1DO@JMHGPCHG@?$AAR?$AAx?$AA_?$AAI?$AAn?$AAt?$AAe?$AAr?$AAr?$AAu?$AAp?$AAt?$AA_?$AAT?$AAr?$AAi?$AAg?$AAg?$AAe?$AAr@ 10001820     ConfigParser.obj
 0001:00000860       ??_C@_1DO@HONDFPK@?$AAT?$AAx?$AA_?$AAI?$AAn?$AAt?$AAe?$AAr?$AAr?$AAu?$AAp?$AAt?$AA_?$AAT?$AAr?$AAi?$AAg?$AAg?$AAe?$AAr@ 10001860     ConfigParser.obj
 0001:000008a0       ??_C@_1DO@JOMMLPNE@?$AAT?$AAx?$AA_?$AAI?$AAn?$AAt?$AAe?$AAr?$AAr?$AAu?$AAp?$AAt?$AA_?$AAT?$AAr?$AAi?$AAg?$AAg?$AAe?$AAr@ 100018a0     ConfigParser.obj
 0001:000008e0       ??_C@_1BO@CLLBHNOO@?$AAF?$AAl?$AAo?$AAw?$AA_?$AAO?$AAf?$AAf?$AA_?$AAL?$AAe?$AAv?$AAe?$AAl?$AA?$AA@ 100018e0     ConfigParser.obj
 0001:00000900       ??_C@_1BM@FKEALHLG@?$AAF?$AAl?$AAo?$AAw?$AA_?$AAO?$AAn?$AA_?$AAL?$AAe?$AAv?$AAe?$AAl?$AA?$AA@ 10001900     ConfigParser.obj
 0001:00000920       ??_C@_1EA@FCDBIJCN@?$AAR?$AAe?$AAc?$AAe?$AAi?$AAv?$AAe?$AA_?$AAI?$AAn?$AAt?$AAe?$AAr?$AAr?$AAu?$AAp?$AAt?$AA_?$AAT?$AAr@ 10001920     ConfigParser.obj
 0001:00000960       ??_C@_1EC@JOHHNGND@?$AAT?$AAr?$AAa?$AAn?$AAs?$AAm?$AAi?$AAt?$AA_?$AAI?$AAn?$AAt?$AAe?$AAr?$AAr?$AAu?$AAp?$AAt?$AA_?$AAT@ 10001960     ConfigParser.obj
 0001:000009a4       ??_C@_1BI@GEBICGMH@?$AAF?$AAi?$AAf?$AAo?$AA_?$AAL?$AAe?$AAv?$AAe?$AAl?$AAs?$AA?$AA@ 100019a4     ConfigParser.obj
 0001:000009bc       ??_C@_1CE@FHCKENKN@?$AAC?$AAr?$AAy?$AAs?$AAt?$AAa?$AAl?$AA_?$AAF?$AAr?$AAe?$AAq?$AAu?$AAe?$AAn?$AAc?$AAy?$AA?$AA@ 100019bc     ConfigParser.obj
 0001:000009e0       ??_C@_15GANGMFKL@?$AA?$CF?$AAs?$AA?$AA@ 100019e0     ConfigParser.obj
 0001:000009e8       ??_C@_1M@MNHBCACD@?$AAT?$AAi?$AAt?$AAl?$AAe?$AA?$AA@ 100019e8     ConfigParser.obj
 0001:000009f4       ??_C@_1CE@EOJPOKCA@?$AAA?$AAp?$AAp?$AAl?$AAi?$AAc?$AAa?$AAt?$AAi?$AAo?$AAn?$AA_?$AAT?$AAi?$AAt?$AAl?$AAe?$AA?$AA@ 100019f4     ConfigParser.obj
 0001:00000a18       ??_C@_1BI@MHELFDAB@?$AA?2?$AAW?$AAi?$AAn?$AAd?$AAo?$AAw?$AAs?$AA?2?$AA?$CF?$AAs?$AA?$AA@ 10001a18     ConfigParser.obj
 0001:00000a30       ??_C@_15JJPIMNBO@?$AAr?$AAb?$AA?$AA@ 10001a30     ConfigParser.obj
 0001:00000a98       DllEntry                   10001a98 f   buspcie950.obj
 0001:00000b34       Deinit                     10001b34 f   buspcie950.obj
 0001:00000df4       Init                       10001df4 f   buspcie950.obj
 0001:000023a0       _tfsubstring               100033a0 f   ConfigParser.obj
 0001:000023ec       ?_ffeosubsec@@YAHPAXQAG@Z  100033ec f   ConfigParser.obj
 0001:00002438       ?ValidateCrystalFrequency@@YAHH@Z 10003438 f   ConfigParser.obj
 0001:00002560       ?ValidateValues@@YAXPAU_CONFIG_DATA_@@@Z 10003560 f   ConfigParser.obj
 0001:00002698       ?_textractValue@@YAPAGPAG@Z 10003698 f   ConfigParser.obj
 0001:000026d8       ParseConfigFile            100036d8 f   ConfigParser.obj
 0001:00002e08       BusTransBusAddrToStatic    10003e08 f   ceddk:CEDDK.dll
 0001:00002e18       BusTransBusAddrToVirtual   10003e18 f   ceddk:CEDDK.dll
 0001:00002e28       CreateBusAccessHandle      10003e28 f   ceddk:CEDDK.dll
 0001:00002e38       KernelLibIoControl         10003e38 f   coredll:COREDLL.dll
 0001:00002e48       EventModify                10003e48 f   coredll:COREDLL.dll
 0001:00002e58       DisableThreadLibraryCalls  10003e58 f   coredll:COREDLL.dll
 0001:00002e68       InterruptDone              10003e68 f   coredll:COREDLL.dll
 0001:00002e78       InterlockedExchange        10003e78 f   coredll:COREDLL.dll
 0001:00002e88       WaitForSingleObject        10003e88 f   coredll:COREDLL.dll
 0001:00002e98       CloseHandle                10003e98 f   coredll:COREDLL.dll
 0001:00002ea8       DeactivateDevice           10003ea8 f   coredll:COREDLL.dll
 0001:00002eb8       wcstoul                    10003eb8 f   coredll:COREDLL.dll
 0001:00002ec8       RegQueryValueExW           10003ec8 f   coredll:COREDLL.dll
 0001:00002ed8       RegSetValueExW             10003ed8 f   coredll:COREDLL.dll
 0001:00002ee8       wcslen                     10003ee8 f   coredll:COREDLL.dll
 0001:00002ef8       ActivateDeviceEx           10003ef8 f   coredll:COREDLL.dll
 0001:00002f08       RegCreateKeyExW            10003f08 f   coredll:COREDLL.dll
 0001:00002f18       CreateThread               10003f18 f   coredll:COREDLL.dll
 0001:00002f28       InterruptInitialize        10003f28 f   coredll:COREDLL.dll
 0001:00002f38       CreateEventW               10003f38 f   coredll:COREDLL.dll
 0001:00002f48       LoadIntChainHandler        10003f48 f   coredll:COREDLL.dll
 0001:00002f58       wcschr                     10003f58 f   coredll:COREDLL.dll
 0001:00002f68       wcsstr                     10003f68 f   coredll:COREDLL.dll
 0001:00002f78       wsprintfW                  10003f78 f   coredll:COREDLL.dll
 0001:00002f88       RegEnumKeyExW              10003f88 f   coredll:COREDLL.dll
 0001:00002f98       RegCloseKey                10003f98 f   coredll:COREDLL.dll
 0001:00002fa8       free                       10003fa8 f   coredll:COREDLL.dll
 0001:00002fb8       malloc                     10003fb8 f   coredll:COREDLL.dll
 0001:00002fc8       wcstol                     10003fc8 f   coredll:COREDLL.dll
 0001:00002fd8       RegOpenKeyExW              10003fd8 f   coredll:COREDLL.dll
 0001:00002fe8       wcscpy                     10003fe8 f   coredll:COREDLL.dll
 0001:00002ff8       memcpy                     10003ff8 f   coredll:COREDLL.dll
 0001:00003008       fgetws                     10004008 f   coredll:COREDLL.dll
 0001:00003018       wcscmp                     10004018 f   coredll:COREDLL.dll
 0001:00003028       wcsrchr                    10004028 f   coredll:COREDLL.dll
 0001:00003038       fclose                     10004038 f   coredll:COREDLL.dll
 0001:00003048       _wtol                      10004048 f   coredll:COREDLL.dll
 0001:00003058       feof                       10004058 f   coredll:COREDLL.dll
 0001:00003068       _wfopen                    10004068 f   coredll:COREDLL.dll
 0001:00003078       swprintf                   10004078 f   coredll:COREDLL.dll
 0001:00003088       __IMPORT_DESCRIPTOR_CEDDK  10004088     ceddk:CEDDK.dll
 0001:0000309c       __IMPORT_DESCRIPTOR_COREDLL 1000409c     coredll:COREDLL.dll
 0001:000030b0       __NULL_IMPORT_DESCRIPTOR   100040b0     ceddk:CEDDK.dll
 0002:00000000       __imp_BusTransBusAddrToVirtual 10005000     ceddk:CEDDK.dll
 0002:00000004       __imp_CreateBusAccessHandle 10005004     ceddk:CEDDK.dll
 0002:00000008       __imp_BusTransBusAddrToStatic 10005008     ceddk:CEDDK.dll
 0002:0000000c       \177CEDDK_NULL_THUNK_DATA  1000500c     ceddk:CEDDK.dll
 0002:00000010       __imp_KernelLibIoControl   10005010     coredll:COREDLL.dll
 0002:00000014       __imp_EventModify          10005014     coredll:COREDLL.dll
 0002:00000018       __imp_DisableThreadLibraryCalls 10005018     coredll:COREDLL.dll
 0002:0000001c       __imp_InterruptDone        1000501c     coredll:COREDLL.dll
 0002:00000020       __imp_InterlockedExchange  10005020     coredll:COREDLL.dll
 0002:00000024       __imp_WaitForSingleObject  10005024     coredll:COREDLL.dll
 0002:00000028       __imp_CloseHandle          10005028     coredll:COREDLL.dll
 0002:0000002c       __imp_DeactivateDevice     1000502c     coredll:COREDLL.dll
 0002:00000030       __imp_wcstoul              10005030     coredll:COREDLL.dll
 0002:00000034       __imp_RegQueryValueExW     10005034     coredll:COREDLL.dll
 0002:00000038       __imp_RegSetValueExW       10005038     coredll:COREDLL.dll
 0002:0000003c       __imp_wcslen               1000503c     coredll:COREDLL.dll
 0002:00000040       __imp_ActivateDeviceEx     10005040     coredll:COREDLL.dll
 0002:00000044       __imp_RegCreateKeyExW      10005044     coredll:COREDLL.dll
 0002:00000048       __imp_CreateThread         10005048     coredll:COREDLL.dll
 0002:0000004c       __imp_InterruptInitialize  1000504c     coredll:COREDLL.dll
 0002:00000050       __imp_CreateEventW         10005050     coredll:COREDLL.dll
 0002:00000054       __imp_LoadIntChainHandler  10005054     coredll:COREDLL.dll
 0002:00000058       __imp_wcschr               10005058     coredll:COREDLL.dll
 0002:0000005c       __imp_wcsstr               1000505c     coredll:COREDLL.dll
 0002:00000060       __imp_wsprintfW            10005060     coredll:COREDLL.dll
 0002:00000064       __imp_RegEnumKeyExW        10005064     coredll:COREDLL.dll
 0002:00000068       __imp_RegCloseKey          10005068     coredll:COREDLL.dll
 0002:0000006c       __imp_free                 1000506c     coredll:COREDLL.dll
 0002:00000070       __imp_malloc               10005070     coredll:COREDLL.dll
 0002:00000074       __imp_wcstol               10005074     coredll:COREDLL.dll
 0002:00000078       __imp_RegOpenKeyExW        10005078     coredll:COREDLL.dll
 0002:0000007c       __imp_wcscpy               1000507c     coredll:COREDLL.dll
 0002:00000080       __imp_memcpy               10005080     coredll:COREDLL.dll
 0002:00000084       __imp_fgetws               10005084     coredll:COREDLL.dll
 0002:00000088       __imp_wcscmp               10005088     coredll:COREDLL.dll
 0002:0000008c       __imp_wcsrchr              1000508c     coredll:COREDLL.dll
 0002:00000090       __imp_fclose               10005090     coredll:COREDLL.dll
 0002:00000094       __imp__wtol                10005094     coredll:COREDLL.dll
 0002:00000098       __imp_feof                 10005098     coredll:COREDLL.dll
 0002:0000009c       __imp__wfopen              1000509c     coredll:COREDLL.dll
 0002:000000a0       __imp_swprintf             100050a0     coredll:COREDLL.dll
 0002:000000a4       \177COREDLL_NULL_THUNK_DATA 100050a4     coredll:COREDLL.dll
 0002:000000a8       dpCurSettings              100050a8     buspcie950.obj
 0002:00000500       m_pDispatchThread          10005500     buspcie950.obj
 0002:00000580       Pcie950BusInfo             10005580     <common>

 entry point at        0001:00000a98

 Static symbols

 0001:00000ab0       BusIstThread               10001ab0 f   buspcie950.obj
 0001:00000bf8       ReadKeyList                10001bf8 f   buspcie950.obj
 0001:00000cfc       ReadKeyDword               10001cfc f   buspcie950.obj
 0001:00000d58       WriteKeyDword              10001d58 f   buspcie950.obj
 0001:00000d9c       WriteKeyString             10001d9c f   buspcie950.obj
